:100000000C94CD010C94FE010C94FE010C94FE01A5
:100010000C94FE010C94FE010C94FE010C94FE0164
:100020000C94FE010C94FE010C94FE010C94FE0154
:100030000C94FE010C94FE010C94FE010C94FE0144
:100040000C94FE010C94FE010C94FE010C94FE0134
:100050000C94FE010C94FE010C94FE010C94AD1066
:100060000C94FE010C9483100C9459100C94FE0116
:100070000C94FE010C94FE010C94FE010C94FE0104
:100080000C94FE010C94FE010C94FE010C94FE01F4
:100090000C942F100C9405100C94FE010C94FE018E
:1000A0000C94FE010C94FE010C94FE010C94FE01D4
:1000B0000C94FE010C94FE010C94FE010C94FE01C4
:1000C0000C94FE010C94FE010C94FE010C94DB0FC9
:1000D0000C94B10F0C94FE010C94FE010C94FE01E3
:1000E0000C94FE010C946F070C94BD160C947C04C8
:1000F0000C94DB0D0C94A7020C9446040C94BD07E1
:100100000C943F070C94F60D0C94E40D0C941E1502
:100110000C944B0E0C943E020C94B70D0C944E06AE
:100120000C9477040C94ED0D0C944E030C947A14FB
:100130000C9461040C9407150C945E170C94B50292
:100140000C94CA0D0C9471060C9447160C9465041B
:100150000C944A040C942F0E0C9475160C945B04AA
:100160000C94C10D0C944E040C9421150C9428068B
:100170000C9442040C9485070C948C170C94460E36
:100180000C9457040C94210E0C949A150C94F710AF
:100190000C94C9070C9420060C9493020C94D30D74
:1001A0000C9452160C94F5050C9467060C948F066B
:1001B0000C94090E0C94B8140C9445070C94370E4B
:1001C0000C94AB140C9484020C94F1070C948104ED
:1001D0000C94D6140C9485060C94FF0D0C94D31536
:1001E0000C9447170C9430060C94130E0C94FD05D8
:1001F0000C947B060C9401030C949F070C941A0E2C
:100200000C9430150C945D070C9416060C9444065F
:100210000C944F070C9469040C943A060C940C0649
:100220000C94BA160C9451040C9402060C946F04AE
:100230000C94280E0C947D040C94410E0C943C04F8
:100240000C945D060C947304000021002400270028
:100250002A002D00300033000101000004010701D5
:100260000A0100002200250028002B002E0031008A
:10027000340002010000050108010B01000020000C
:100280002300260029002C002F003200000100006E
:100290000301060109010505050507050808080809
:1002A000020202020A0A080804040404010101010E
:1002B0000101010103030303030303030407070709
:1002C0000C0C0C0C0C0C0C0C0202020206060606AE
:1002D000060606060B0B0B0B0B0B0B0B0A0A0A0A86
:1002E0000A0A08080707050505040404010210208E
:1002F000200808102040102040800201020108045C
:1003000002010102040810204080804020100804EF
:100310000201800402018040201008040201080448
:10032000020101020408102040800102040810208C
:100330004080040810204080048008100440801091
:10034000204000000A0B02090C0D0E0807030401EF
:10035000000000000000000000000000000000009D
:10036000000000000000000000000000000012116A
:10037000100000000000000000000000000000006D
:10038000000000000000000000000000000000006D
:100390000000000000000000F71011241FBECFEF86
:1003A000D1E2DEBFCDBF00E00CBF13E0A0E0B2E0C1
:1003B000E2E3F7E300E00BBF02C007900D92AC341C
:1003C000B107D9F726E0ACE4B3E001C01D92AA3032
:1003D000B207E1F711E0CDECD1E000E006C02197D3
:1003E0000109802FFE010E948F1BCC3CD10780E0C9
:1003F0000807A9F70E9470110C94971B0C94000039
:100400000F931F93CF93DF93EC019A01AB01E8891F
:10041000F98982E08083EC85FD8510820E851F8539
:1004200060E874E88EE190E00E940E1921503109D5
:10043000410951095695479537952795F80120832D
:10044000188EEC89FD8986E08083EA89FB898081AA
:1004500080618083EA89FB89808188608083EA8962
:10046000FB89808180688083EA89FB8980818F7D18
:100470008083DF91CF911F910F910895AF92BF922A
:10048000CF92DF92EF92FF920F931F93CF93DF9360
:100490006C017B018B01040F151FEB015E01AE188F
:1004A000BF08C017D10759F06991D601ED91FC91B1
:1004B0000190F081E02DC6011995892B79F7C501CE
:1004C000DF91CF911F910F91FF90EF90DF90CF9030
:1004D000BF90AF900895FC01A089B1898C91A68945
:1004E000B78982FD0FC09C91818D8F5F8F73228DA4
:1004F000821749F0A18DAE0FBF2FB11D5D969C9361
:10050000818F08958C910895FC01538D448D252F82
:1005100030E0842F90E0821B930B541710F0CF969D
:10052000089501970895FC01918D828D981761F0CF
:10053000A28DAE0FBF2FB11D5D968C91928D9F5FE6
:100540009F73928F90E008958FEF9FEF0895FC01C5
:10055000918D828D981731F0828DE80FF11D858D78
:1005600090E008958FEF9FEF0895FC01918D228D0B
:10057000892F90E0805C9F4F821B91098F73992790
:10058000089583E394E00E94B50221E0892B09F4E9
:1005900020E0822F089580ED94E00E94B50221E0D2
:1005A000892B09F420E0822F08958DE695E00E94C2
:1005B000B50221E0892B09F420E0822F0895FC0187
:1005C000A48DA80FB92FB11DA35ABF4F2C91848DB4
:1005D00090E001968F739927848FA689B7892C9311
:1005E000A089B1898C91837080648C93938D848D64
:1005F000981306C00288F389E02D80818F7D808367
:100600000895EF92FF920F931F93CF93DF93EC0126
:1006100081E0888F9B8D8C8D98131AC0E889F989A9
:10062000808185FF15C09FB7F894EE89FF896083AC
:10063000E889F98980818370806480839FBF81E02D
:1006400090E0DF91CF911F910F91FF90EF9008956F
:10065000F62E0B8D10E00F5F1F4F0F731127E02E4A
:100660008C8D8E110CC00FB607FCFACFE889F98982
:10067000808185FFF5CFCE010E94DF02F1CFEB8DA7
:10068000EC0FFD2FF11DE35AFF4FF0829FB7F89456
:100690000B8FEA89FB8980818062CFCFCF93DF9374
:1006A000EC01888D8823B9F0AA89BB89E889F9898A
:1006B0008C9185FD03C0808186FD0DC00FB607FCBF
:1006C000F7CF8C9185FFF2CF808185FFEDCFCE01F2
:1006D0000E94DF02E9CFDF91CF910895EF92FF9260
:1006E0001F93CF93DF9380918A03811168C080911B
:1006F0007603811164C011E083E394E00E94B502A7
:1007000004970CF45CC080917603811158C083E398
:1007100094E00E94A702892B59F083E394E00E94A1
:10072000A702429729F083E394E00E949302E4CF6A
:1007300083E394E00E949302D82F80938C0383E399
:1007400094E00E94930280938D0383E394E00E94DF
:100750009302C82F80938E0383E394E00E94930258
:1007600080938F0399279C012C5F3F4F3093750333
:10077000209374030297439780F4DD2311F0D23164
:1007800061F4C03141F0C53431F08C2F8D7F883455
:1007900011F0CC3411F4109376038091760381111B
:1007A000ABCF83E394E00E94930280917203909117
:1007B0007303019690937303809372039DCF80918E
:1007C0008A03811135C080917603882389F183E300
:1007D00094E00E94B502E0907403F09075039701D5
:1007E000245031098217930718F114E0C12FD0E08B
:1007F000CE15DF0548F483E394E00E949302C457CA
:10080000DC4F88831F5FF2CF83E394E00E94B50240
:10081000892B29F083E394E00E949302F5CF84E0D2
:1008200080938A03109276031092730310927203DE
:10083000DF91CF911F91FF90EF9008958150823109
:1008400008F05AC0E82FF0E08827E65DFB4F8F4F95
:100850000C948F1B4A044E043C04420446047C045E
:10086000510457045B046104650469046F04730454
:100870007C0477047D048104809180008F778093CD
:1008800080000895809180008F7DF9CF8091800055
:10089000877FF5CF84B58F7784BD089584B58F7D2C
:1008A000FBCF8091B0008F778093B0000895809146
:1008B000B0008F7DF9CF809190008F77809390006A
:1008C0000895809190008F7DF9CF80919000877F6F
:1008D000F5CF8091A0008F778093A000089580913C
:1008E000A0008F7DF9CF8091A000877FF5CF809108
:1008F00020018F77809320010895809120018F7DC2
:10090000F9CF80912001877FF5CFCF93DF93282FF8
:1009100030E0F901EE5BFC4F8491F901E451FD4FA9
:10092000D491F901EA56FD4FC491CC23A1F0811175
:100930000E941E04EC2FF0E0EE0FFF1FE458FD4F65
:10094000A591B491EC91ED2381E090E009F480E071
:10095000DF91CF91089580E090E0FACF1F93CF937D
:10096000DF93282F30E0F901EE5BFC4F8491F90111
:10097000E451FD4FD491F901EA56FD4FC491CC23C7
:10098000A9F0162F81110E941E04EC2FF0E0EE0F4B
:10099000FF1FEE59FD4FA591B4918FB7F894EC91DC
:1009A000111108C0D095DE23DC938FBFDF91CF916A
:1009B0001F910895DE2BF8CFCF93DF9380918B03A7
:1009C000823009F44DC0833009F465C081112FC015
:1009D00080ED94E00E94B50203974CF180ED94E025
:1009E0000E94A7028E37910581F580ED94E00E9468
:1009F000930280ED94E00E94930280ED94E00E94C7
:100A0000A702079739F480ED94E00E94930282E0F8
:100A100080938B0380ED94E00E94A7024D9751F4E0
:100A200080ED94E00E94930283E080938B03DF913A
:100A3000CF91089580ED94E00E94B502892BB9F31F
:100A400080ED94E00E949302F5CF80ED94E00E9447
:100A5000B502892B61F380ED94E00E949302F5CFFB
:100A600080ED94E00E94B50208970CF3C8E0D8E04E
:100A700080ED94E00E949302D0938B03C150C1F7A4
:100A800080ED94E00E94B502892B89F280ED94E01C
:100A90000E949302F5CF61E08AE10E94AE0480EDEE
:100AA00094E00E94B5024E9714F2CEE1D4E080EDBE
:100AB00094E00E949302D0938B03C150C1F780ED64
:100AC00094E00E94B502892B09F4B1CF80ED94E047
:100AD0000E949302F4CF80E090E0892B29F00E94DD
:100AE000D50281110E9400000E94CB0281110E9458
:100AF000DC040E94C10281110E946E0380E090E03C
:100B0000892B49F080E090E0892B29F00E940000B9
:100B100081110C9400000895CF93DF9390E0FC01C5
:100B2000E451FD4F24918A569D4FFC018491882306
:100B3000D1F090E0880F991FFC01E85BFD4FA59173
:100B4000B491FC01EE59FD4FC591D49161110EC0D5
:100B50009FB7F8948C91E22FE0958E238C93288197
:100B6000E223E8839FBFDF91CF9108958FB7F89478
:100B7000EC91E22BEC938FBFF6CF1F93CF93DF93D3
:100B8000182FEB0161E00E948C05209739F460E09A
:100B9000812FDF91CF911F910C94AE04CF3FD105EF
:100BA00011F461E0F5CFE12FF0E0EE5BFC4FE49152
:100BB000E150E23108F0B3C0F0E08827ED51FA4F80
:100BC0008F4F0C948F1BF505FD0502060C061606CB
:100BD0008F062006280630063A0644064E065D06B5
:100BE00067068F0671067B06850684B5806884BD1E
:100BF000C7BDDF91CF911F91089584B5806284BDF8
:100C0000C8BDF7CF80918000806880938000D0932A
:100C10008900C0938800EDCF80918000806280932E
:100C20008000D0938B00C0938A00E3CF8091800036
:100C3000886080938000D0938D00C0938C00D9CFC2
:100C40008091B00080688093B000C093B300D1CF92
:100C50008091B00080628093B000C093B400C9CF8F
:100C600080919000806880939000D0939900C09309
:100C70009800BFCF80919000806280939000D093C5
:100C80009B00C0939A00B5CF8091900088608093BC
:100C90009000D0939D00C0939C00ABCF8091A000AA
:100CA00080688093A0008091A0008F7B8093A0003B
:100CB000D093A900C093A8009CCF8091A00080622F
:100CC0008093A000D093AB00C093AA0092CF8091F4
:100CD000A00088608093A000D093AD00C093AC00CA
:100CE00088CF80912001806880932001D0932901D2
:100CF000C09328017ECF80912001806280932001E3
:100D0000D0932B01C0932A0174CF80912001886079
:100D100080932001D0932D01C0932C016ACFC0385D
:100D2000D1050CF03ECF33CF863308F086532091A7
:100D30007B00982F9870277F922B90937B00877071
:100D4000806480937C0080917A00806480937A0034
:100D500080917A0086FDFCCF809178009091790097
:100D600008953FB7F8948091800390918103A091FA
:100D70008203B091830326B5A89B05C02F3F19F0CD
:100D80000196A11DB11D3FBFBA2FA92F982F88270B
:100D9000BC01CD01620F711D811D911D43E0660FE5
:100DA000771F881F991F4A95D1F708958091E60310
:100DB0009091E703A091E803B091E903813E9E4240
:100DC000A105B10520F089E080937E0309C08091E0
:100DD000FC039091FD0380359105C0F410927E03D1
:100DE000E0917E03EA3008F002C1F0E08827E45089
:100DF000F94F8F4F0C948F1BF1073F0745074F07A3
:100E00005D076F0785079F07C907BD079C01205530
:100E100031092436310510F481E0D6CF9C01245BE2
:100E200031092436310510F482E0CECF9C012851DF
:100E300031402436310510F483E0C6CF9C012C5795
:100E400031402436310510F484E0BECF9C01205E91
:100E500031402436310510F485E0B6CF9C0124548E
:100E600032402436310510F486E0AECF885A9240E5
:100E70008436910510F487E0A7CF88E0A5CF61E024
:100E800085E20E94AE0460E005C061E085E20E9458
:100E9000AE0461E084E20E94AE0460E009C061E05B
:100EA00085E20E94AE0461E084E20E94AE0461E04B
:100EB00083E20E94AE0460E00DC061E085E20E9422
:100EC000AE0461E084E20E94AE0461E083E20E942D
:100ED000AE0461E082E20E94AE0460E011C061E015
:100EE00085E20E94AE0461E084E20E94AE0461E00B
:100EF00083E20E94AE0461E082E20E94AE0461E0FF
:100F000081E20E94AE0460E015C061E085E20E94CB
:100F1000AE0461E084E20E94AE0461E083E20E94DC
:100F2000AE0461E082E20E94AE0461E081E20E94D0
:100F3000AE0461E080E20E94AE0460E019C061E0AE
:100F400085E20E94AE0461E084E20E94AE0461E0AA
:100F500083E20E94AE0461E082E20E94AE0461E09E
:100F600081E20E94AE0461E080E20E94AE0461E092
:100F70008FE10E94AE0460E029C080917C039091D3
:100F80007D03833091052CF5019690937D0380932A
:100F90007C0361E085E20E94AE0461E084E20E948D
:100FA000AE0461E083E20E94AE0461E082E20E944E
:100FB000AE0461E081E20E94AE0461E080E20E9442
:100FC000AE0461E08FE10E94AE0461E08EE10C941A
:100FD000AE04863091053CF4019690937D03809396
:100FE0007C0360E04DCF10927D0310927C03089546
:100FF00060E089E00E94AE0480918503843009F4AA
:1010000063C030F4882381F0813091F10C94D606CE
:10101000863009F47EC008F475C08730B9F71092A5
:10102000F10310928503F2CF8091E3038130D1F078
:10103000809126044091FC035091FD0320912904E6
:1010400030912A04840F952F911D2817390708F431
:10105000C901883C910510F488EC90E090937B03E3
:1010600080937A0381E0809385038093E303CECF5E
:101070008091FC039091FD0320917A0330917B03D2
:1010800028173907D8F02091290430912A0428170D
:101090003907A0F080910A0490910B04883E934098
:1010A00068F48091E6039091E703A091E803B09182
:1010B000E903803E9E42A105B10520F085E08093C2
:1010C0008503A4CF84E0FBCF609115046093D8031F
:1010D0008091FC039091FD0320917A0330917B0372
:1010E0002817390740F02091290430912A0470E034
:1010F0002817390710F470E060E085E00E94BD0514
:1011000087E0DDCF70E060E085E00E94BD0586E00D
:10111000D6CF70E060E085E00E94BD058091790344
:1011200090911604891740F087E080938503109210
:10113000E303109279036ACF8F5F8093790366CFC0
:1011400070E060E085E00E94BD05809184038130FD
:1011500099F030F0823031F18630E1F10C94D6060E
:101160008091E303813031F48093840382E08093A3
:10117000E303F4CF82E0F8CF61E089E00E94AE049F
:1011800080917803909117048917E8F060E089E076
:101190000E94AE041092F1031092780386E08093CF
:1011A0008403DCCF61E089E00E94AE048091780383
:1011B0002091FC033091FD03283C310540F09091D3
:1011C0001804891718F78F5F80937803C7CF909121
:1011D0001904DACF8091770390911604891738F0BB
:1011E0001092F1031092840310927703B7CF8F5FB0
:1011F00080937703B3CFDB01EC91F0E0E050FE4F3A
:10120000E081E927F0E0E050FE4F908189278C9340
:101210000895FC0101900020E9F73197AF01481BC8
:10122000590BBC018DE695E00C943E028F929F9283
:10123000AF92BF920F931F93CF93DF93CDB7DEB7DB
:10124000A1970FB6F894DEBF0FBECDBF19A24230F2
:1012500008F44AE08E010F5D1F4F842E912CB12CB3
:10126000A12CA50194010E940E19E62FB901CA0113
:10127000EA30F4F4E05DD801EE938D01232B242BAA
:10128000252B79F790E080E0109719F0CD010E94AE
:101290000909A1960FB6F894DEBF0FBECDBFDF914E
:1012A000CF911F910F91BF90AF909F908F90089515
:1012B000E95CE1CFEF92FF920F931F93CF93DF93FF
:1012C0007C018B010E94F818D82FD801EC91F0E036
:1012D000E050FE4FE081C82FCE27CC93C701019686
:1012E0000E94F818EC2FF0E0E050FE4F9081982714
:1012F000F80190832D2F30E0322F2227820F932F79
:10130000911DDF91CF911F910F91FF90EF90089564
:10131000CF93DF931F921F92CDB7DEB71A8281E081
:101320008983BE016F5F7F4F90E080E00E945A0981
:101330008230910508F060C190932C0480932B04B7
:10134000BE016F5F7F4F82E090E00E945A098533B3
:1013500023E0920708F055C190932A048093290452
:10136000BE016F5F7F4F84E090E00E945A09853391
:1013700023E0920708F048C1909328048093270443
:10138000BE016F5F7F4F86E090E00E945A099FEF99
:10139000980F983C08F03DC180932604BE016F5F12
:1013A0007F4F88E090E00E945A09873222E092073E
:1013B00008F031C19093250480932404BE016F5F2F
:1013C0007F4F8AE090E00E945A09873222E092071C
:1013D00008F024C19093230480932204BE016F5F20
:1013E0007F4F8CE090E00E945A09893823E19207F0
:1013F00008F017C19093210480932004BE016F5F11
:101400007F4F8EE090E00E945A09893823E19207CD
:1014100008F00AC190931F0480931E04BE016F5F01
:101420007F4F80E190E00E945A09893522E09207BF
:1014300008F0FDC090931D0480931C04BE016F5FF3
:101440007F4F82E190E00E945A09893522E092079D
:1014500008F0F0C090931B0480931A04BE016F5FE4
:101460007F4F84E190E00E945A09853608F0E5C07C
:1014700080931904BE016F5F7F4F86E190E00E9468
:101480005A098B3008F0DBC080931804BE016F5FEF
:101490007F4F88E190E00E945A09853108F0D1C061
:1014A00080931704BE016F5F7F4F8AE190E00E9436
:1014B0005A09853608F0C7C080931604BE016F5FD5
:1014C0007F4F8CE190E00E945A0980931504BE0181
:1014D0006F5F7F4F8EE190E00E945A09813127E2D1
:1014E000920708F0B2C09093140480931304BE01D5
:1014F0006F5F7F4F80E290E00E945A099093120440
:1015000080931104BE016F5F7F4F82E290E00E94E2
:101510005A099093100480930F04BE016F5F7F4FB0
:1015200084E290E00E945A0990930E0480930D0487
:10153000E981F0E0E050FE4F80818983BE016E5F5B
:101540007F4F86E290E00E945A099981981709F42A
:101550004CC010922C0410922B0426E232E03093FF
:101560002A0420932904109228041092270492E35D
:101570009093260444EF51E05093250440932404B3
:10158000509323044093220448E755E050932104EC
:101590004093200448E057E050931F0440931E04FA
:1015A00030931D0420931C0428EC30E030931B047E
:1015B00020931A0494E19093190492E090931804F4
:1015C0009AE0909317049EE19093160490E590930F
:1015D000150420ED37E0309314042093130428E918
:1015E0003AE3309312042093110480930C040F907B
:1015F0000F90DF91CF91089510922C0410922B043C
:101600009FCE86E292E0A8CE109228041092270482
:10161000B7CE82E3C1CE84EF91E0CCCE84EF91E0EF
:10162000D9CE88E795E0E6CE88E097E0F3CE86E273
:1016300092E000CF88EC90E00DCF84E119CF82E0FA
:1016400023CF88E02DCF8EE137CF80ED97E04BCFD1
:10165000FF920F931F93CF93DF93F82E8B01EA0134
:10166000E881F0E0E050FE4F808189278883692F70
:10167000C8010E940019E881F0E0E050FE4F80812F
:101680008F2588836F2DC8010196DF91CF911F911F
:101690000F91FF900C940019CF93DF931F92CDB759
:1016A000DEB781E08983AE014F5F5F4F70E060E09D
:1016B00080912B0490912C040E94280BAE014F5F67
:1016C0005F4F62E070E08091290490912A040E94AB
:1016D000280BAE014F5F5F4F64E070E080912704FC
:1016E000909128040E94280B80912604AE014F5F40
:1016F0005F4F66E070E090E00E94280BAE014F5F04
:101700005F4F68E070E080912404909125040E946E
:10171000280BAE014F5F5F4F6AE070E080912204BA
:10172000909123040E94280BA895AE014F5F5F4F54
:101730006CE070E080912004909121040E94280BBD
:10174000AE014F5F5F4F6EE070E080911E0490919C
:101750001F040E94280BAE014F5F5F4F60E170E0F5
:1017600080911C0490911D040E94280BAE014F5FD4
:101770005F4F62E170E080911A0490911B040E9417
:10178000280B80911904AE014F5F5F4F64E170E058
:1017900090E00E94280BA89580911804AE014F5F3D
:1017A0005F4F66E170E090E00E94280B8091170483
:1017B000AE014F5F5F4F68E170E090E00E94280B40
:1017C00080911604AE014F5F5F4F6AE170E090E0D8
:1017D0000E94280B80911504AE014F5F5F4F6CE1B2
:1017E00070E090E00E94280BAE014F5F5F4F6EE10A
:1017F00070E080911304909114040E94280BAE01B4
:101800004F5F5F4F60E270E080911104909112048D
:101810000E94280BA895AE014F5F5F4F62E270E017
:1018200080910F04909110040E94280BAE014F5F2D
:101830005F4F64E270E080910D0490910E040E946D
:10184000280BE981F0E0E050FE4F80818983AE01F2
:101850004F5F5F4F66E270E090E00E94280B0F90B0
:10186000DF91CF910895CF938091E503882321F0F4
:101870008091E40381110DC0809171039091160451
:10188000981798F481E08093E5038093E403109225
:10189000710380918A038130E9F058F08430C9F1F6
:1018A000853009F43BC2CF9108958F5F8093710317
:1018B000F0CF60E089E10E94AE0460E08AE10E941E
:1018C000AE0460E08CE10E94AE0460E08DE1CF9157
:1018D0000C94AE04809189038F5F823018F480935A
:1018E0008903E1CF1092890361E089E10E94AE048F
:1018F00060E08AE10E94AE0410928A0383E394E0E0
:101900000E94B502892B79F283E394E00E9493024E
:10191000F5CF2091740330917503B90162507109BC
:10192000FB01E457FC4F808190E0982F88272557D2
:101930003C4FD9012C91820F911D50E040E0E0E036
:101940002E2F30E02617370740F424573C4FD9019B
:101950002C91420F511DEF5FF3CF8417950709F0CB
:10196000C7C1C0918C03CC2311F0C23159F48091CE
:101970008E03883409F498C170F4803101F1853404
:1019800009F4BEC061E089E10E94AE0461E08AE131
:101990000E94AE0481C08A3409F499C18C3491F755
:1019A00060E089E10E94AE0461E08AE10E94AE0439
:1019B000C23109F071C081E0809388036DC060E09E
:1019C00089E10E94AE0461E08AE10E94AE04809148
:1019D000900390E0982F882720919103820F911D0A
:1019E0009093DE038093DD0380919203282F30E0F3
:1019F000322F222780919303820F932F911D909372
:101A0000CD038093CC039C0120553109293131400D
:101A100008F048C034E6389FA001399F500D1124CA
:101A20005093CD034093CC038091940390E0982F82
:101A3000882720919503820F911D389FA001399F1F
:101A4000500D11245093CF034093CE0380919A03FD
:101A500090E0982F882740919B03480F592F511DE4
:101A6000EFE080919C0390E0982F882720919D03C0
:101A7000820F911DE89FB001E99F700D1124E49F32
:101A80009001E59F300D11242617370708F49B01BC
:101A90003093E0032093DF0385E080938A03109264
:101AA000890301CF80549F4181369D46A8F78091DC
:101AB000940390E0982F882720919503820F911D21
:101AC0009093CF038093CE0360919A03862F90E08A
:101AD000982F882760919B03680F792F711D90E0E4
:101AE00080E00E94521A20E030E040EC5FE30E9468
:101AF000091B0E94231A7093E0036093DF03CCCF8D
:101B000060E089E10E94AE0461E08AE10E94AE04D7
:101B1000C23111F681E08093870320919103822FD7
:101B200090E0982F882720919203280F392F311D9C
:101B3000E0919003ED51E33108F5F0E08827EC5592
:101B4000F24F8F4F0C948F1BB70DC10DCA0DD30DE3
:101B5000DB0DE40DED0DF60DFF0D090E130E1A0E43
:101B6000210E280E2F0E370E410E460E4B0E223040
:101B7000310520F430932C0420932B040E944C0B4D
:101B80008BCF2533F3E03F07C8F730932A04209327
:101B90002904F4CF253343E0340780F73093280439
:101BA00020932704EBCFC9010197883C910530F7BA
:101BB00020932604E3CF273282E03807F8F63093EB
:101BC000250420932404DACF2732A2E03A07B0F6A6
:101BD0003093230420932204D1CF2938B3E13B076B
:101BE00068F63093210420932004C8CF2938E3E11C
:101BF0003E0720F630931F0420931E04BFCF2935E3
:101C0000F2E03F0708F0BACF30931D0420931C0484
:101C1000B5CF293542E0340708F0B0CF30931B042C
:101C200020931A04ABCF2536310508F0A7CF2093B7
:101C30001904A4CF2B30310508F0A0CF209318044D
:101C40009DCF2531310508F099CF2093170496CF09
:101C50002536310508F092CF209316048FCF2F3F01
:101C6000310511F008F08ACF2093150487CF213178
:101C700087E2380708F082CF3093140420931304CE
:101C80007DCF309312042093110478CF3093100449
:101C900020930F0473CF2436310508F46FCF3093AF
:101CA0000E0420930D046ACF60E089E10E94AE0427
:101CB00061E08AE10E94AE04C23109F0EDCE81E01C
:101CC0008093E5031092E40380938603E5CE60E001
:101CD00089E10E94AE0461E08AE10E94AE04C23153
:101CE00009F0DACE1092E50381E08093E403ECCFB3
:101CF00061E089E10E94AE0460E08AE10E94AE04E6
:101D000010928A0383E394E00E94B502892B09F4C0
:101D1000CACD83E394E00E949302F4CF309187030D
:101D20008091880381114AC03111E2C010924C03A6
:101D300082E180934D0380E180934E0387E080939E
:101D40004F038091FC039091FD0390935003809387
:101D500051038091F003809352038091EA038093B2
:101D600053038091E20380935403ECE4F3E090E0AA
:101D700080E020E03191830F911D2F5F2930D1F752
:101D8000909355038093560361E08CE10E94AE046A
:101D900061E08DE10E94AE0440914F0350E04C5F42
:101DA0005F4F6CE473E083E394E00E943E02109284
:101DB0008A0383E394E00E944E0383CD10924C0388
:101DC00082E180934D038CE480934E0381E2809303
:101DD0004F0380912B0480935003809129049091AC
:101DE0002A04909351038093520380912704909189
:101DF0002804909353038093540380912604809386
:101E00005503809124049091250490935603809368
:101E10005703809122049091230490935803809358
:101E20005903809120049091210490935A03809348
:101E30005B0380911E0490911F0490935C03809338
:101E40005D0380911C0490911D0490935E03809328
:101E50005F0380911A0490911B0490936003809318
:101E60006103809119048093620380911804809328
:101E70006303809117048093640380911604809318
:101E800065038091150480936603809113049091FB
:101E900014049093670380936803809111049091D8
:101EA00012049093690380936A0380910F049091C8
:101EB000100490936B0380936C0380910D049091B8
:101EC0000E0490936D0380936E03ECE4F3E090E0D6
:101ED00080E020E04191840F911D2F5F2332D1F7E4
:101EE00090936F038093700310928803332309F15A
:101EF00010924C0382E180934D0382E480934E0361
:101F000084E080934F031092500386E58093510341
:101F1000ECE4F3E090E080E020E03191830F911D4C
:101F20002F5F2630D1F79093520380935303109282
:101F3000870380918603882309F426CF10924C03EF
:101F400082E180934D0382E480934E0382E080938C
:101F50004F031092500386E580935103109286033D
:101F600013CF1F920F920FB60F9211240BB60F9240
:101F70002F933F934F935F936F937F938F939F9391
:101F8000AF93BF93EF93FF9383E394E00E94DF024C
:101F9000FF91EF91BF91AF919F918F917F916F9141
:101FA0005F914F913F912F910F900BBE0F900FBEFD
:101FB0000F901F9018951F920F920FB60F92112439
:101FC0000BB60F922F933F934F935F936F937F9333
:101FD0008F939F93AF93BF93EF93FF9383E394E02B
:101FE0000E946B02FF91EF91BF91AF919F918F91F2
:101FF0007F916F915F914F913F912F910F900BBE09
:102000000F900FBE0F901F9018951F920F920FB652
:102010000F9211240BB60F922F933F934F935F9320
:102020006F937F938F939F93AF93BF93EF93FF93A0
:1020300080ED94E00E94DF02FF91EF91BF91AF919C
:102040009F918F917F916F915F914F913F912F91D0
:102050000F900BBE0F900FBE0F901F9018951F9200
:102060000F920FB60F9211240BB60F922F933F933E
:102070004F935F936F937F938F939F93AF93BF9390
:10208000EF93FF9380ED94E00E946B02FF91EF913C
:10209000BF91AF919F918F917F916F915F914F9180
:1020A0003F912F910F900BBE0F900FBE0F901F907E
:1020B00018951F920F920FB60F9211240BB60F9224
:1020C0002F933F934F935F936F937F938F939F9340
:1020D000AF93BF93EF93FF938DE695E00E94DF02ED
:1020E000FF91EF91BF91AF919F918F917F916F91F0
:1020F0005F914F913F912F910F900BBE0F900FBEAC
:102100000F901F9018951F920F920FB60F921124E7
:102110000BB60F922F933F934F935F936F937F93E1
:102120008F939F93AF93BF93EF93FF938DE695E0CB
:102130000E946B02FF91EF91BF91AF919F918F91A0
:102140007F916F915F914F913F912F910F900BBEB7
:102150000F900FBE0F901F9018951F920F920FB601
:102160000F9211242F933F938F939F93AF93BF931D
:102170008091C8039091C903A091CA03B091CB0389
:1021800030917F0326E0230F2D3758F50296A11DCD
:10219000B11D20937F038093C8039093C903A0933C
:1021A000CA03B093CB038091800390918103A091E7
:1021B0008203B09183030196A11DB11D809380031A
:1021C00090938103A0938203B0938303BF91AF9157
:1021D0009F918F913F912F910F900FBE0F901F9065
:1021E000189529E8230F0396A11DB11DD2CFE3E373
:1021F000F4E01382128248EE53E060E070E0448322
:1022000055836683778384E093E09183808325ED13
:1022100030E03587248724ED30E03787268720EDAE
:1022200030E0318B208B21ED30E0338B228B22ED9F
:1022300030E0358B248B26ED30E0378B268B118EEA
:10224000128E138E148EE0EDF4E01382128244831A
:10225000558366837783918380832DEC30E03587C7
:1022600024872CEC30E03787268728EC30E0318B50
:10227000208B29EC30E0338B228B2AEC30E0358B3D
:10228000248B2EEC30E0378B268B118E128E138E22
:10229000148EEDE6F5E01382128244835583668343
:1022A00077839183808385EC90E09587848784ECA5
:1022B00090E09787868780EC90E0918B808B81EC13
:1022C00090E0938B828B82EC90E0958B848B86ECF4
:1022D00090E0978B868B118E128E138E148E08953C
:1022E000CF93DF931F92CDB7DEB7789484B5826029
:1022F00084BD84B5816084BD85B5826085BD85B5AA
:10230000816085BD80916E00816080936E00109227
:1023100081008091810082608093810080918100A2
:102320008160809381008091800081608093800033
:102330008091B10084608093B1008091B000816091
:102340008093B00080919100826080939100809191
:1023500091008160809391008091900081608093D2
:1023600090008091A10082608093A1008091A100E3
:1023700081608093A1008091A00081608093A00083
:1023800080912101826080932101809121018160EF
:1023900080932101809120018160809320018091B0
:1023A0007A00846080937A0080917A0082608093C2
:1023B0007A0080917A008E7F80937A0080917A00F3
:1023C000806880937A001092C10010922E041092BF
:1023D000D4031092D5031092D6031092D703109213
:1023E0002F04109230041092310410923204109293
:1023F000C6031092C703279A15B860E086E10E94D1
:102400008C0560E087E10E948C0560E088E10E9415
:102410008C0540E855E260E070E08DE695E00E94B2
:10242000000240E855E260E070E080ED94E00E9438
:10243000000240E855E260E070E083E394E00E942F
:102440000002789461E089E00E948C0561E085E0FB
:102450000E948C0561E085E20E948C0561E084E2C7
:102460000E948C0561E083E20E948C0561E082E2BB
:102470000E948C0561E081E20E948C0561E080E2AF
:102480000E948C0561E08FE10E948C0561E08EE185
:102490000E948C058091B100887F81608093B1009B
:1024A00080919100887F8160809391001092F10368
:1024B00010928503109284031092D0031092D103DE
:1024C0001092D2031092D3031092D9031092DA0320
:1024D0001092DB031092DC031092EF031092E303DF
:1024E0001092E6031092E7031092E8031092E903BA
:1024F00061E089E10E948C0561E08AE10E948C051F
:1025000061E08CE10E948C0561E08DE10E948C0508
:1025100010928B0310928A03109289031092880301
:102520001092870381E08093E5038093E403109287
:10253000860340E855E260E070E083E394E00E94A7
:1025400000020E9488090E9488090E944C0BA895ED
:10255000ECE8F3E084EB93E011928E179F07E1F72C
:1025600083E394E00E94B502892B29F083E394E091
:102570000E949302F5CF40E052EC61E070E08DE6FE
:1025800095E00E94000282E193E00E94090986E240
:1025900093E00E9409090E94B1064B015C01E0E151
:1025A000CE2EE7E2DE2EE12CF12C0E94B106681956
:1025B00079098A099B09683E734081059105A8F352
:1025C00021E0C21AD108E108F10838EE830E33E0A9
:1025D000931EA11CB11CC114D104E104F10429F71C
:1025E00084E991E090930E0480930D040E944C0BBB
:1025F00089E293E00E9409096091290470912A04FC
:1026000090E080E00E94521A2AE037ED43E25CE35A
:102610000E94091B6B017C01AC019B010E94761B8F
:10262000882309F4A7C08FE393E00E94090986E29A
:1026300093E00E94090940E1942E5AE0852E64E659
:10264000E62EF12C76ECC72E73E0D72E0E94B10651
:1026500000912F0410913004209131043091320404
:10266000601771078207930708F4B9C52B013C0175
:10267000401A510A620A730A93018201003117421B
:102680002105310508F48FC160932F047093300445
:1026900080933104909332047090C7030091C60375
:1026A00010E058015FEFA51AB50A87E0A822BB2405
:1026B000000F111F36E0432E82E0471408F4D6C005
:1026C0000E949406F801EA54FC4F91838083A09203
:1026D000C60373947092C7038091FE0381110BC0EF
:1026E0008091FC039091FD039093FB038093FA0388
:1026F00081E08093FE038091F203811103C081E0A9
:102700008093F203E091F103EC3208F031C1F0E084
:102710008827E257FC4E8F4F0C948F1B7A14AB1412
:10272000D61407151E15B814B814B814B814B81474
:1027300021153015B814B814B8149A15D315B81457
:10274000B814B814471652167516B814B814B8143D
:10275000B814B814B814B814BA16B814B814B81415
:10276000B814B814B814B814B814B814BD16471770
:102770005E178C172FEF3FEF4FE75FE7C701B601FA
:102780000E94761B81110DC02FEF3FEF4FE75FE7EF
:10279000C701B6010E94AC1918161CF483E493E03B
:1027A00044CF2FEF3FEF4FE75FE4C701B6010E9430
:1027B000041B18161CF487E493E037CF2FEF3FEF8C
:1027C0004FE75FECC701B6010E94AC1987FDF3CF5C
:1027D0002AE037ED43EA5BE3C701B6010E944019E6
:1027E0004B015C010E94231A6B017C010E94521A6A
:1027F0009B01AC01C501B4010E943F194B015C0172
:102800004AE0C701B6010E9416096EE28DE695E026
:102810000E94010320E030E040E251E4C501B40130
:102820000E94091B4B015C010E94231A6B01F12CD1
:10283000E12C4AE0C701B6010E941609C701B601A2
:102840000E94521A9B01AC01C501B4010E943F19BC
:1028500020E030E040E251E40E94091B0E94231A6C
:1028600090E080E04AE00E941609E1CE0E949406C2
:10287000F801EA54FC4F91838083A092C6036091D3
:10288000B4037091B503E6EBF3E081919191680F89
:10289000791FCE16DF06C9F793E0769567959A956E
:1028A000E1F76C39710548F41092FD031092FC03B6
:1028B0001092B5031092B4030FCF90E080E00E9415
:1028C000521A27E03FE548E15CE30E94091B2DEC2A
:1028D0003CEC4CE85FE30E943F1920E030E048EC1C
:1028E00052E40E94091B0E94231A7093FD03609317
:1028F000FC03DECF80910804811127C060E089E0ED
:102900000E94AE0481E08093F1031092F0031092D4
:10291000EF031092EB031092EC031092ED03109270
:10292000EE038091FC039091FD038834934050F0B6
:1029300070E060E085E00E94BD050E94A0088FE085
:102940008093EA030E94D60613C08092F1038FEFB2
:102950008093F003E6CF0E94D60682E08093F103D5
:102960001092E6031092E7031092E8031092E90335
:102970008091FC039091FD039093FB038093FA03F5
:1029800080912E04813009F423C408F4D1C282302E
:1029900009F4F1C2833009F418C380912E048F5FCB
:1029A000837080932E040E946B0550CE1091070413
:1029B000111108C070E060E085E00E94BD0583E071
:1029C0008093F10380910604811104C084E0809318
:1029D000F103CECF813061F6113051F68091E503DD
:1029E000882371F08091E403882381F370E060E034
:1029F00085E00E94BD051092E3031092F103B8CF69
:102A000070E060E085E00E94BD0583E0E0CF2091AA
:102A1000FC033091FD0380912704909128048217D4
:102A2000930718F40E94A008A3CF1092F10360E06E
:102A300089E00E94AE041092EA039ACF0E94F80740
:102A400097CF8091E20381110BC08091070481111F
:102A500030C01092E10370E060E085E00E94BD05A7
:102A60008091DF039091E003892B09F061C0809190
:102A7000DD039091DE038035910508F059C0809107
:102A8000EF038F3F81F58EE18093F1031092EB030A
:102A90001092EC031092ED031092EE038091E1038B
:102AA0008F3F09F065CF8FE08093F1031092EF0321
:102AB0005FCF8091060481110CC08FEF8093E103FA
:102AC0001092EB031092EC031092ED031092EE03C0
:102AD000C7CF8091E503882309F4BBCF8091E4033D
:102AE000882359F3BDCF8091EB039091EC03A09123
:102AF000ED03B091EE030196A11DB11D8093EB0390
:102B00009093EC03A093ED03B093EE031092F103C6
:102B1000409113045091140470E060E0841795070D
:102B2000A607B70708F4BACF84E18093F103B6CFC4
:102B300088E2FBCF60E089E00E94AE042FB7F894F2
:102B40008091C8039091C903A091CA03B091CB03AF
:102B50002FBF8093D9039093DA03A093DB03B09344
:102B6000DC038091290490912A040A972091FC03A8
:102B70003091FD032817390760F46091D80370E0A5
:102B800085E00E94BD0580EF8093EA039092F103F7
:102B9000D9CE70E060E085E00E94BD051092EA03A6
:102BA0001092F103CFCE8FB7F8944090C8035090A5
:102BB000C9036090CA037090CB038FBF4092D403C7
:102BC0005092D5036092D6037092D7030E94D60626
:102BD0008091E503882311F1809107048823F1F0A7
:102BE0008091D9039091DA03A091DB03B091DC03CB
:102BF000481659066A067B0618F1B301A201481B64
:102C0000590B6A0B7B0B8091110490911204B0E078
:102C1000A0E0481759076A077B0790F04092D90354
:102C20005092DA036092DB037092DC0370E060E0A4
:102C300085E00E94BD051092EA031092E103DDCE0B
:102C40006091FC037091FD038091290490912A0406
:102C50000A96853333E0930710F084E393E0681716
:102C6000790740F070E060E085E00E94BD05909239
:102C7000F1037ECE90E080E04AE00E94160986E2F1
:102C800093E00E9409096091150470E0EDCF70E0B7
:102C900060E085E00E94BD051092E20385E180932B
:102CA000F10350CE61E089E00E94AE042FB7F894A2
:102CB0008091C8039091C903A091CA03B091CB033E
:102CC0002FBF8093D0039093D103A093D203B093EE
:102CD000D30382E08093E30386E18093F1030E94B3
:102CE000D6068FE08093EA0343CE8FB7F8944090E6
:102CF000C8035090C9036090CA037090CB038FBF84
:102D00004092D4035092D5036092D6037092D703B9
:102D10000E94D6068091D0039091D103A091D20356
:102D2000B091D303481659066A067B06F8F0A30152
:102D30009201281B390B4A0B5B0BDA01C901803465
:102D40009F41A105B10590F04092D0035092D1036C
:102D50006092D2037092D30360E089E00E94AE04D7
:102D60008FEF8093EF031092F103BBCF86E1809346
:102D7000F103B7CF1092F1035ECE8FEF8093E203A1
:102D80001092EF03A090CE03B090CF030091CC033C
:102D90001091CD0370E060E085E00E94BD05609079
:102DA000DD037090DE03E091DF03F091E00380919A
:102DB0002404909125046816790610F580911E046C
:102DC00090911F048E179F07D8F0C501B7010E948C
:102DD0007B1B9B01C801B7010E947B1BDB010E948A
:102DE00030191B012C0120911C0430911D04A4E614
:102DF000B0E00E9430196215730584059505A8F4AA
:102E000080912B0490912C04892B91F58AE2809378
:102E1000F103EF2B09F496CD1092EB031092EC0323
:102E20001092ED031092EE038DCD20911A04309193
:102E30001B04A4E6B0E00E943019261637064806A7
:102E40005906C0F48091200490912104E817F907F5
:102E500088F480912204909123046816790650F436
:102E6000309741F080912B0490912C04892B71F6BE
:102E700089E2CDCF8091E403882341F28091E5037C
:102E80008823B1F31092F1031092EA03C2CF10929B
:102E9000E6031092E7031092E8031092E9032091F1
:102EA000FC033091FD038091270490912804821740
:102EB000930708F0BACD0E94A00813CF8091E603D3
:102EC0009091E703A091E803B091E903813E4EE2BF
:102ED0009407A105B105E0F42091290430912A045A
:102EE0002A5031094091FC035091FD0342175307CA
:102EF00078F40196A11DB11D8093E6039093E7033A
:102F0000A093E803B093E9030E94F80780EFEACEAC
:102F10008BE28093F1038FCD1092F10370E060E0BB
:102F200085E00E94BD051092E2030E94D60683CD83
:102F30000091090410E0000F111F86E10E94850432
:102F40008095909581709927082B009309040111B1
:102F50000DC01092080488E10E9485048093070444
:102F600087E10E9485048093060417CD0F3F99F7EF
:102F700000930804F0CF81E00E94940683E00E9451
:102F80009406BC0190E080E00E94521A23E333E3F0
:102F900043E55BE30E94091B20E030E048EC52E48B
:102FA0000E94091B20E030E048EC51E40E94B11976
:102FB0002AE037ED43E25CE30E94B1190E94231A34
:102FC00070930B0460930A04E8CC81E08983A0909D
:102FD0002B04B0902C04BE016F5F7F4FC5010E948F
:102FE000FB088091290490912A0412E0853353E074
:102FF000950730F411E022E0A216B10408F410E0C5
:10300000BE016F5F7F4F0E94FB0880912704909163
:103010002804853333E0930708F013E0BE016F5FA7
:103020007F4F0E94FB08809126049FEF980F983CE9
:1030300008F014E0BE016F5F7F4F90E00E94FB0834
:103040008091240490912504873242E0940708F08F
:1030500015E0BE016F5F7F4F0E94FB088091220444
:1030600090912304873252E0950708F016E0BE01E4
:103070006F5F7F4F0E94FB08809120049091210494
:10308000893823E1920708F017E0BE016F5F7F4F98
:103090000E94FB0880911E0490911F04893833E13F
:1030A000930708F018E0BE016F5F7F4F0E94FB0896
:1030B00080911C0490911D04893542E0940708F02A
:1030C00019E0BE016F5F7F4F0E94FB0880911A04D8
:1030D00090911B04893552E0950708F01AE0BE0173
:1030E0006F5F7F4F0E94FB0880911904853608F0BE
:1030F0001BE0BE016F5F7F4F90E00E94FB08809154
:1031000018048B3008F01CE0BE016F5F7F4F90E029
:103110000E94FB0880911704853108F01DE0BE0174
:103120006F5F7F4F90E00E94FB0880911604853608
:1031300008F01EE0BE016F5F7F4F90E00E94FB0829
:1031400080911504BE016F5F7F4F90E00E94FB08E5
:103150008091130490911404813127E2920708F0C2
:1031600010E1BE016F5F7F4F0E94FB08BE016F5FE1
:103170007F4F80911104909112040E94FB08BE01C0
:103180006F5F7F4F80910F04909110040E94FB08A5
:1031900080910D0490910E048436910508F413E19A
:1031A000BE016F5F7F4F0E94FB08E981F0E0E050B5
:1031B000FE4F908180910C04981301C011110E9460
:1031C000880980912D04893130F010922D041F9AC6
:1031D0000E94330CE2CB8F5F80932D04F9CF1092C5
:1031E0002F04109230041092310410923204DBCB81
:1031F000F999FECF92BD81BDF89A992780B50895BF
:10320000262FF999FECF1FBA92BD81BD20BD0FB602
:10321000F894FA9AF99A0FBE01960895A1E21A2E2F
:10322000AA1BBB1BFD010DC0AA1FBB1FEE1FFF1F6A
:10323000A217B307E407F50720F0A21BB30BE40BBA
:10324000F50B661F771F881F991F1A9469F7609501
:103250007095809590959B01AC01BD01CF010895BB
:10326000A29FB001B39FC001A39F700D811D1124C7
:10327000911DB29F700D811D1124911D089550580C
:10328000BB27AA270E9457190C94CA1A0E94BC1A7D
:1032900038F00E94C31A20F039F49F3F19F426F445
:1032A0000C94B91A0EF4E095E7FB0C94B31AE92FCD
:1032B0000E94DB1A58F3BA17620773078407950751
:1032C00020F079F4A6F50C94FD1A0EF4E0950B2E7F
:1032D000BA2FA02D0B01B90190010C01CA01A00168
:1032E0001124FF27591B99F0593F50F4503E68F1C3
:1032F0001A16F040A22F232F342F4427585FF3CF04
:10330000469537952795A795F0405395C9F77EF4D4
:103310001F16BA0B620B730B840BBAF09150A1F01D
:10332000FF0FBB1F661F771F881FC2F70EC0BA0FA3
:10333000621F731F841F48F4879577956795B7952B
:10334000F7959E3F08F0B0CF9395880F08F0992726
:10335000EE0F9795879508950E948F1A08F481E0E3
:1033600008950E94C5190C94CA1A0E94C31A58F0F5
:103370000E94BC1A40F029F45F3F29F00C94B31A64
:1033800051110C94FE1A0C94B91A0E94DB1A68F3BE
:103390009923B1F3552391F3951B550BBB27AA270E
:1033A00062177307840738F09F5F5F4F220F331F48
:1033B000441FAA1FA9F335D00E2E3AF0E0E832D010
:1033C00091505040E695001CCAF72BD0FE2F29D013
:1033D000660F771F881FBB1F261737074807AB07E5
:1033E000B0E809F0BB0B802DBF01FF2793585F4F5A
:1033F0003AF09E3F510578F00C94B31A0C94FE1AE3
:103400005F3FE4F3983ED4F3869577956795B7953B
:10341000F7959F5FC9F7880F911D9695879597F946
:103420000895E1E0660F771F881FBB1F62177307BF
:103430008407BA0720F0621B730B840BBA0BEE1FD4
:1034400088F7E09508950E94E31A88F09F5798F056
:10345000B92F9927B751B0F0E1F0660F771F881F99
:10346000991F1AF0BA95C9F714C0B13091F00E94B3
:10347000FD1AB1E008950C94FD1A672F782F882764
:10348000B85F39F0B93FCCF3869577956795B395DA
:10349000D9F73EF490958095709561957F4F8F4F49
:1034A0009F4F0895E89409C097FB3EF4909580954E
:1034B000709561957F4F8F4F9F4F9923A9F0F92FFA
:1034C00096E9BB279395F695879577956795B79578
:1034D000F111F8CFFAF4BB0F11F460FF1BC06F5F5E
:1034E0007F4F8F4F9F4F16C0882311F096E911C070
:1034F000772321F09EE8872F762F05C0662371F091
:1035000096E8862F70E060E02AF09A95660F771FA4
:10351000881FDAF7880F9695879597F90895990F80
:103520000008550FAA0BE0E8FEEF16161706E8078D
:10353000F907C0F012161306E407F50798F0621BAE
:10354000730B840B950B39F40A2661F0232B242B83
:10355000252B21F408950A2609F4A140A6958FEFA2
:10356000811D811D089597F99F6780E870E060E0F4
:1035700008959FEF80EC089500240A94161617060C
:1035800018060906089500240A9412161306140654
:1035900005060895092E0394000C11F4882352F0B7
:1035A000BB0F40F4BF2B11F460FF04C06F5F7F4F6F
:1035B0008F4F9F4F089557FD9058440F551F59F056
:1035C0005F3F71F04795880F97FB991F61F09F3F10
:1035D00079F087950895121613061406551FF2CF39
:1035E0004695F1DF08C0161617061806991FF1CF89
:1035F00086957105610508940895E894BB276627B0
:103600007727CB0197F908950E948F1A08F48FEF5E
:1036100008950E941C1B0C94CA1A0E94BC1A38F010
:103620000E94C31A20F0952311F00C94B31A0C9445
:10363000B91A11240C94FE1A0E94DB1A70F3959F9C
:10364000C1F3950F50E0551F629FF001729FBB2799
:10365000F00DB11D639FAA27F00DB11DAA1F649F35
:103660006627B00DA11D661F829F2227B00DA11DE8
:10367000621F739FB00DA11D621F839FA00D611D6E
:10368000221F749F3327A00D611D231F849F600D8F
:10369000211D822F762F6A2F11249F5750409AF0B8
:1036A000F1F088234AF0EE0FFF1FBB1F661F771F44
:1036B000881F91505040A9F79E3F510580F00C940F
:1036C000B31A0C94FE1A5F3FE4F3983ED4F3869548
:1036D00077956795B795F795E7959F5FC1F7FE2BAF
:1036E000880F911D9695879597F908950E948F1AD6
:1036F000880B990B0895AA1BBB1B51E107C0AA1F99
:10370000BB1FA617B70710F0A61BB70B881F991F82
:103710005A95A9F780959095BC01CD010895EE0FBB
:10372000FF1F881F8BBF0790F691E02D1994F89426
:02373000FFCFC9
:1037320000316253C4F5A697B988DBEA7D4C1F2E8F
:103742004372211087B6E5D4FACB98A93E0F5C6D7F
:1037520086B7E4D5427320113F0E5D6CFBCA99A86F
:10376200C5F4A796013063527C4D1E2FB889DAEB5F
:103772003D0C5F6EF9C89BAA84B5E6D7407122134F
:103782007E4F1C2DBA8BD8E9C7F6A594033261503F
:10379200BB8AD9E87F4E1D2C02336051C6F7A4952F
:1037A200F8C99AAB3C0D5E6F4170231285B4E7D61F
:1037B2007A4B1829BE8FDCEDC3F2A190073665540F
:1037C20039085B6AFDCC9FAE80B1E2D344752617FF
:1037D200FCCD9EAF38095A6B4574271681B0E3D2EF
:1037E200BF8EDDEC7B4A192806376455C2F3A091DF
:1037F2004776251483B2E1D0FECF9CAD3A0B5869CF
:1038020004356657C0F1A293BD8CDFEE79481B2ABE
:10381200C1F0A3920534675678491A2BBC8DDEEFAE
:1038220082B3E0D1467724153B0A5968FFCE9DAC9E
:103832000000000001033E0284024E03B50293021F
:10384200A7025265736574212076657273696F6E83
:1038520020342E3034000D0A005072657373696F84
:103862006E206D6178205B6261725D203D20006E8A
:0C387200616E00696E66006F76660000F3
:00000001FF
